:040000008A11442DF0
:100A1E0064008001840A0406031900340406102DB4
:100A2E0001308312031386008A11FC258A1164306B
:100A3E008A115C258A1108007E088A007F088200D0
:100A4E0023258A118000840A04087D0603190034C8
:100A5E00FF0A0319FE0A272DF400740883120313EC
:100A6E0086008A11AD258A110D30F5000130F50290
:100A7E00031D422D432D3D2D0800F801F901FA0109
:100A8E0083134030840051308A110F258A11403073
:100A9E00FD000530FE008D30FF00203084008A11ED
:100AAE0027258A1183018A118B2EF0000430F20063
:100ABE005330F1000130F102031D662D672D612DBB
:100ACE000130F202031D6C2D6D2D5F2D0130F002F1
:100ADE00031D722D732D5D2D0800F20003100030E2
:100AEE0003180130F100721C7D2D7E2D822D7308AE
:100AFE00F0007008F1070310F30D0310F20CF2086A
:100B0E00031D8A2D8B2D7A2D710808003034313457
:100B1E00323433343434353436343734383439347B
:100B2E00413442344334443445344634EE34ED34A7
:100B3E00EB34E734DE34DD34DB34D734BE34BD344D
:100B4E00BB34B7347E347D347B347734F914790872
:100B5E008312031385001130F3000130F302031DDD
:100B6E00B92DBA2DB42D7915790885001130F20002
:100B7E000130F202031DC42DC52DBF2DFB30F00038
:100B8E007008F905790885001130F1000130F10285
:100B9E00031DD22DD32DCD2D0800031000300318C8
:100BAE000130FA007A08303E84008313000878067C
:100BBE00031DE22DE32DEA2D7A08203E8400000865
:100BCE0083120313CF007A08013EFA0010307A0226
:100BDE00031CF22DF32DD92D831203134F0886001B
:100BEE0064308A115C258A110800FD30F00070080F
:100BFE00F90579088312031385001130F3000130D3
:100C0E00F302031D0B2E0C2E062E79157908850086
:100C1E001130F2000130F202031D162E172E112E86
:100C2E00FB30F0007008F905790885001130F100ED
:100C3E000130F102031D242E252E1F2E0800F03048
:100C4E00831603138600831203130608CC004C0888
:100C5E00F039CB0078080F39F80078084B04F8000B
:100C6E000608CC004C08F039CB004B08F03A0319BB
:100C7E00412E422E432E372E031000300318013022
:100C8E008316031386008A11D4258A118312031347
:100C9E004F08CE00CD010314CD0D0800F600023032
:100CAE008312031386008A11FC258A1164308A117F
:100CBE005C258A112830F30076088A1174258A1172
:100CCE00F40077087407F6000310003003180130A3
:100CDE00F700842E14308312031386008A11FC252C
:100CEE008A112130F5000130F502031D7F2E802E72
:100CFE007A2E0130F4007408F70776087702031C89
:100D0E00892E8A2E712E08009813031000300318B6
:100D1E000130831603139B0007309C000310003034
:100D2E00031801309D0003100030031801308500B8
:100D3E0083120313051003100030031801308316BD
:100D4E000313860032308A115C258A118A112A27F4
:100D5E008A118A1117258A110310003003180130E9
:100D6E00F70000308A1155268A118A11C9268A1178
:100D7E0083120313CA004A088A1133258A11BC2E26
:100D8E008A11002803100030031801308312031358
:100D9E00CD000310003003180130831603138500B5
:100DAE00F0308600811303100030031801308312D7
:100DBE0003138500EF30F800780886000430C90070
:100DCE00232F7808F500F6017508D1007608D200B9
:100DDE000230D3000030D4008A118E278A1183137B
:100DEE00831203135108F800780886000A308A111E
:100DFE005C258A1183120313061E062F072F132F4D
:100E0E00861E0A2F0B2F132F061F0E2F0F2F132F99
:100E1E00861B122F132F162F8A1126268A11831244
:100E2E0003134D08013A031D1D2F1E2F202F4E08B0
:100E3E00292F4908FF3EC900C908031D272F282F57
:100E4E00E82EC92E080038308312031386008A114B
:100E5E00FC258A1132308A115C258A1138308312B2
:100E6E00031386008A11FC258A1121308312031385
:100E7E00D4000130D402031D452F462F402F3830A9
:100E8E0086008A11FC258A11213083120313D500A6
:100E9E000130D502031D542F552F4F2F38308600A9
:100EAE008A11FC258A11213083120313D3000130DD
:100EBE00D302031D632F642F5E2F013086008A112B
:100ECE00FC258A1132308A115C258A110D3083126D
:100EDE00031386008A11FC258A1121308312031315
:100EEE00D1000130D102031D7D2F7E2F782F0630C9
:100EFE0086008A11FC258A11213083120313D20039
:100F0E000130D202031D8C2F8D2F872F0800031066
:100F1E00003003180130F20083120313D41F982FF0
:100F2E00992FA12FD309D409D30A0319D40AF20198
:100F3E000314F20DD21FA42FA52FAE2FD109D20963
:100F4E00D10A0319D20A0130F0007008F2060030FF
:100F5E00F3000030F400540853040319B72FB82FD0
:100F6E00F02FF1010314F10DC72F01300310D30D33
:100F7E00D40DFF3E031DBD2F0130F0007008F107A8
:100F8E00D41FCA2FCB2FBC2F01300310F30DF40D3D
:100F9E00FF3E031DCC2F54085202031DD82F5308B9
:100FAE005102031CDB2FDC2FE32F5308D102540810
:100FBE00031CD203D202731401300310D40CD30CD1
:100FCE00FF3E031DE42F0130F102031DEF2FF02F22
:100FDE00CB2F7208031DF42FF92FF309F409F30A2E
:100FEE000319F40A7408D201D2077308D101D1078C
:020FFE000800E9
:00000001FF
